:020000000F28C7
:10000800FE00030EF1000408F2000A08F300831250
:100018007F08F40056287B288B010730831299004B
:10002800703083169F0006309100493083129F007C
:10003800F9308316920005308312920093010C3038
:100048009500850106308316850083128701831683
:10005800870184308100F6017D30F5007508F800CD
:10006800F7010630831281008B168B17F930F500E3
:100078000000F50B3C284028000083129F149F18AD
:1000880043281E08F5007508F600073076020318A5
:1000980051280730F5007508F6007603FF3AFF3E51
:1000A80093003A280B1D70280B110630810001308F
:1000B800F802F808031D68287D30F0007008F80081
:1000C8000430F0007008F700770803196F28013032
:1000D800F7020716702807127408FF0073088A00D1
:1000E80072088400710E8300FE0E7E0E0900F60170
:0600F800F701830110284E
:02400E00E1F3DC
:00000001FF
